:100000005EC578C577C576C575C565CB73C572C540
:1000100071C570C56FC56EC56DC56CC56BC5184221
:100020008124E00729940401F888F80000F8000012
:10003000E8A8B80088A8F8003820F800B8A8E800B8
:10004000F8A8E80008E81800F8A8F800B8A8F80030
:100050001403009F1591009F859F0097959D009325
:10006000940F0000000040CF42CF00CF42CF00CF1E
:1000700046CB00CF08C700C0404004070507000773
:100080000305000701070003040300070504290511
:10009000FE03010101011121418141211101F10101
:1000A00001010101010101010101F1011121418160
:1000B00041211101010103FEFCFF000000000014BA
:1000C00012111011121410FF1010901010101010B7
:1000D000901010FF101412111011121400000000E3
:1000E000FFFFFF0000000000000000000000000013
:1000F000FF000020110A040A11200000FF00000088
:10010000000000000000000000FFFFFF00000040B2
:1001100040E15149494951E141FF4141E1514949DA
:100120004951E14141FF41E15149494951E14040D3
:100130000000FFFF0F1830303030303132323231B2
:1001400030303130303031323232313030303130A5
:1001500030313232323130303030382F1F1902FF17
:10016000010101010101010101010101010101017F
:10017000010101010101FFFE010303030303030366
:10018000030303030303030303030303030303033F
:1001900003000000003800000000003700AE20001F
:1001A000B0C8001040813FA1A6A83FA4D300D5F05D
:1001B000D922DA12DB208D14AF815A245A5080489C
:1001C000200A0112044120448088200C012201826F
:1001D00004308011048001200404200180020608FC
:1001E00000000806020602000808000206000000DF
:1001F000003600020202020202010204081020007E
:1002000000000000000000000000000000000000EE
:1002100000000000000000000000000000000000DE
:10022000000080C0C0E060303030303030303030DE
:10023000303030303030B0703030303030303030FE
:100240003030303030303070B030303030303030EE
:10025000303030303030303060E0C0C080000000DE
:10026000000000000000000000000000000000008E
:10027000000000000000000000000000000000007E
:10028000000000000000000000000000000000006E
:100290000000000000000000000080C0E0F0787C5A
:1002A0005E4F474341404040404040404040404016
:1002B00040404040E05C434040404040404040407F
:1002C0004040404040404040435CE040404040406F
:1002D000404040404040404040404143474F5E7CAA
:1002E00078F0E0C080000000000000000000000086
:1002F00000000000000000000000000000000000FE
:1003000000000000000000000000000000000000ED
:10031000000080C0E0F0783C1E0F070301000000E1
:1003200000000000000000000000000000000000CD
:1003300000C03807000000000000000000000000BE
:1003400000000000000000000000000738C00000AE
:10035000000000000000000000000000000000009D
:1003600000000103070F1E3C78F0E0C08000000091
:10037000000000000000000000000000000000007D
:100380000000000000000000000080C0E0F0783CA9
:100390001E0F07030302020202020202020202020D
:1003A000020202020202020202020202020282723D
:1003B0000E03020202020202020202020202020210
:1003C00002020202020202020202020202030E7290
:1003D000820202020202020202020202020202027D
:1003E000020202020202020202020303070F1E3C83
:1003F00078F0E0C080000000000000000000000075
:1004000000000040E0F0F8FC9E0F07030100000030
:1004100000000000000000000000000000000000DC
:10042000000000000000000000000000E01C0300CD
:1004300000000000000000000000000000000000BC
:1004400000000000000000000000000000000000AC
:10045000031CE0000000000000000000000000009D
:10046000000000000000000000000000000000008C
:1004700000000103070F9EFCF8F0E04000000000C0
:1004800000003F42FC85F9EBABEBEBEBEBEBEBEB6E
:10049000EBEBEBEBEBEBEBEBEBEBEBEBEBEBEBEBAC
:1004A000EBEBEBEBEBEBEBEBEBEBEBE3EBEBEBEBA4
:1004B000EBEBEBEBEBEBEBEBEBEBEBEBEBEBEBEB8C
:1004C000EBEBEBEBEBEBEBEBEBEBEBEBEBEBEBEB7C
:1004D000EBEBEBE3EBEBEBEBEBEBEBEBEBEBEBEB74
:1004E000EBEBEBEBEBEBEBEBEBEBEBEBEBEBEBEB5C
:1004F000EBEBEBEBEBEBABEBF985FC423F0000FEEB
:1005000001FCFEFEFE06D6C6FE067E7EF6EE1EE66A
:10051000FEFEFE76FEFEFEFEFEFEFEFEFEFEFEFE83
:10052000FEFEFEFEFEFEFEFEFEFEFEFEFEFEFEFEEB
:10053000FEFEFEFEFEFEFEFEFEFEFEFC01FE0000D6
:10054000FE01FCFEFEFE067676FE06D6C6FE067EA2
:1005500006FEFEFE76FEFEFEFEFEFEFEFEFEFEFE3B
:10056000FEFEFEFEFEFEFEFEFEFEFEFEFEFEFEFEAB
:10057000FEFEFEFEFEFEFEFEFEFEFEFEFC01FE0395
:1005800004091B2B1B2B1B2B1B2B1B2B1B2B1B2B74
:100590001B2B1B2B1B2B1B2B1B2B1B2B1B2B1B2B2B
:1005A0001B2B3B2B3B2B3B2B3B2B3B2B3B2B3B2B3B
:1005B0003B2B3B2B3B2B3B2B3B2B3B190C070000D6
:1005C0000304091B2B1B2B1B2B1B2B1B2B1B2B1B5C
:1005D0002B1B2B1B2B1B2B1B2B1B2B1B2B1B2B1BEB
:1005E0002B1B2B1B2B3B2B3B2B3B2B3B2B3B2B3B1B
:1005F0002B3B2B3B2B3B2B3B2B3B2B3B190C07006B
:10060000C0E06030B0B0B0B0B0B0B0B0B0B030307A
:100610000000454E4F5F5F5D59585858585D4F4F29
:100620004747000030303030B0B0B0B0B0B0B0307C
:10063000303030000000464F4F4F5D5958585859E0
:100640005D4F4F4F460000003030B0B0B0B0B0B09A
:10065000B0B0B0B03060E0C0000047474F4F5D58C9
:10066000585858595D5F5F4F4E4500C0C0E060303C
:10067000B0B0B03030303030B0B0B0B0B053595806
:10068000484C4C45474747474F5F5D59594060705C
:1006900030B0B0B030303030303030B0B0B030701A
:1006A000005058585D4D4F47474747474F4D5D589D
:1006B000585000B0B0B0B0B03030303030B0B0B022
:1006C0003060E0C0C0604059595D5F4F47474747C1
:1006D000454C4C48585953C0C0E06030B030B03041
:1006E000B030B030B030B030B05349544A554A55AC
:1006F0004A554A554A554A554A45607030B030B05F
:1007000030B030B030B030B030B030700048554A02
:10071000554A554A554A554A554A554A554800B0D2
:1007200030B030B030B030B030B030B03060E0C059
:10073000C060454A554A554A554A554A554A554A50
:1007400054495324384B000000133D7C7C7EFEE668
:10075000E7E3E3E3E3E3E363777F7E3E3E1C0800E9
:1007600000383C7C7E7EFEE6E7E3C3C3C3C3C3E33D
:10077000E7E6FE7E7E7C3C38000000081C3E3E7EA4
:100780007F7763E3E3E3E3E3E3E7E6FE7E7C7C3D40
:10079000130000009ECFC7E36160713333373F1E03
:1007A0001E1E3C3C7E7EF6F6E3E3E3C301C187C038
:1007B000C0E1E3E37377363E3E1C1C1C3E3E3677B9
:1007C00073E3E3E1C0C08700C101C3E3E3E3F6F6EE
:1007D0007E7E3C3C1E1E1E3F373333716061E3C793
:1007E000CF9E9E4FA753A954AA55AA55AA55AA55BC
:1007F000AA55AA55AA55AA55AA550AC18750AA555D
:10080000AA55AA55AA55AA55AA55AA55AA55AA55F0
:10081000AA55AA508700C10A55AA55AA55AA55AA91
:1008200055AA55AA55AA55AA55AA54A953A74F9EE9
:1008300019344E00000000783C9ECEC6E2E2E2F29F
:100840007272723A3A3A3A3A3A3A3A3A3A7AFAF2A8
:10085000F2F2E2E2C2820000000000060F1F1F1F3A
:100860003F3F3F7F7C7878787878787838383C3CA0
:100870003C3E1F1F0F0F070703610000008EC2E2FE
:10088000E2F2F2F2FA7A7A3A3A3A3A3A3A3A3A3AB8
:100890003A3A7A7AFAF2F2F2E2E2C28E000000000C
:1008A0000007070F1F1F3F3F3F7E7C7878787878DE
:1008B0007878787878787C7E3F3F3F1F1F0F070756
:1008C0000000000082C2E2E2F2F2F2FA7A3A3A3A28
:1008D0003A3A3A3A3A3A3A727272F2E2E2E2C6CE00
:1008E0009E3C780000000000610307070F0F1F1FE8
:1008F0003E3C3C3C3838787878787878787C7F3F14
:100900003F3F1F1F1F0F060000000080C0E0F0786F
:100910003C1E0E061A3A3A7A7AFAF2F2E2E2E2C2A1
:10092000C2C2E2E2E2E27272723A3A3A1A1A1A4722
:100930006371707878383C3C1C1C1E0E0E0F070744
:10094000070307070F0F1F1F3E3E7E7C7C787870E1
:1009500000E01C00000E02021A1A3A3A3A7A72F2C9
:10096000F2E2E2E2C2E2E2E2F2F2727A3A3A3A1AEF
:100970001A02020E0000000000707078787C3C3C87
:100980003E1E1E0F0F070707030707070F0F1E1E48
:100990003E3C3C7C787870700000001A1A1A3A3A93
:1009A0003A727272E2E2E2E2C2C2C2E2E2E2F2F25F
:1009B000FA7A7A3A3A1A060E1E3C78F0E0C0801CA9
:1009C000E0007078787C7C7E3E3E1F1F0F0F07078B
:1009D000030707070F0E0E1E1C1C3C3C387878706E
:1009E00071634780C0E0F0783C9E4EA652AA52AA9E
:1009F00052AA52AA52AA52AA52AA52AA52AA52AA17
:100A000052AA52AA52AA12275329542A552A552AC1
:100A1000552A552A552A552A552A552A552A552ADE
:100A2000552A552A552A552A05601C00720E42AADD
:100A300052AA52AA52AA52AA52AA52AA52AA52AAD6
:100A400052AA52AA52AA52AA52AA420E72000000F8
:100A5000502A552A552A552A552A552A552A552AA3
:100A6000552A552A552A552A552A552A552A552A8E
:100A700050000012AA52AA52AA52AA52AA52AA522C
:100A8000AA52AA52AA52AA52AA52AA52AA52A64E8E
:100A90009E3C78F0E0C0801C60052A552A552A55F6
:100AA0002A552A552A552A552A552A552A552A554E
:100AB0002A552A552A552A542953270B2F521124D7
:100AC0001FBECFE5D2E0DEBFCDBF10E0A0E6B0E0B4
:100AD000E6E6FEE102C005900D92A636B107D9F711
:100AE00020E0A6E6B0E001C01D92A138B207E1F710
:100AF0003CD6B7C985CACF92DF92EF92FF920F938F
:100B00001F93CF93DF93362FF801E4903196E49151
:100B1000F12CC42FD0E0C82E880FDD08C701019743
:100B20008C0D9D1D8C179D070CF45EC0CC15DD054A
:100B30000CF45AC0462F660F550B83E05595479528
:100B40008A95E1F7622F70E0641775070CF44CC0CA
:100B50008E2F90E0FC01E40FF51FE617F7070CF469
:100B600043C0B70146D9DC011196241B3770CC195C
:100B7000DD09822F022E000C990BB7013AD9AC0186
:100B8000FE01E80FF91F329680E0AE17BF0748F06C
:100B9000E00FF11F9491892F032E01C0880F0A9452
:100BA000EAF71216C4F44E195F094C0F5D1F4E5F31
:100BB0005F4FF801E40FF51FE491A417B50758F053
:100BC000F0E048E050E0431B510902C0F595E7957D
:100BD0004A95E2F78E2BDF91CF911F910F91FF90F5
:100BE000EF90DF90CF90089580E0F5CFC298C09845
:100BF000C29AC09A089530E020E090E0AC01022E45
:100C000001C0440F0A94EAF747FF0CC0C09AC29A89
:100C1000C2982F5F3F4F2830310581F7C09AC29AA2
:100C2000C2980895C098F3CFC29AC09AC098C2984B
:100C30000895CF93C82FF8DF88E7DDDF80E0DBDFA2
:100C40008C2FD9DFCF91D2CFEFDF88E7D4DF80E4DC
:100C5000D2CFEAEFF1E08491E4EFF1E0E491EE230A
:100C600071F0F0E0EE0FFF1FE351FE4FA591B4913C
:100C7000EC91E82381E090E021F480E0089580E0A9
:100C800090E00895CF93DF9387FF07C08F7769F1D6
:100C9000813069F1823069F183E090E0FC01E75036
:100CA000FE4F24918D509E4FFC0184918823D1F0FA
:100CB00090E0880F991FFC01E956FE4FA591B49171
:100CC000FC01EF56FE4FC591D491611114C09FB73E
:100CD000F8948C91E22FE0958E238C932881E22367
:100CE000E8839FBFDF91CF91089585E0D6CF82E062
:100CF000D4CF84E0D2CF8FB7F894EC91E22BEC9371
:100D00008FBFF0CF8F7787B987B187B9369A369979
:100D1000FECF84B195B10895843028F0883010F06A
:100D200080E008958F5F0895982F81E020917600EC
:100D3000291380E020917700921301C082602091F6
:100D40007800921301C0846020917900921301C051
:100D5000886020917B00921301C0806120917C000B
:100D6000921301C0806220917D00921301C08064C3
:100D700020917E00921301C0806808959F92AF92E7
:100D8000BF92CF92DF92EF92FF920F931F93CF9378
:100D9000DF93A82EC9DFB82ED12CC12C982E9094A9
:100DA0008EE1E82E80E0F82EF601EE5DFF4FC49153
:100DB0004B2D4C2390E080E020E050E0BA01082E5B
:100DC00002C0759567950A94E2F760FD2F5F019662
:100DD0008830910599F7223071F510E000E0E92D97
:100DE000EC23CE2FD0E0CE01002E02C09595879542
:100DF0000A94E2F780FF1AC0802F8EDFE82FF0E020
:100E0000EA58FF4F8081823089F4809169008083A5
:100E1000C1E08C2FDF91CF911F910F91FF90EF9048
:100E2000DF90CF90BF90AF909F9008950F5F1F4FBE
:100E300008301105C1F68FEFC81AD80AE4E0CE16C3
:100E4000D10409F0ADCFD0917A009B2C9094F7019A
:100E500004912B2D202390E080E0C0E030E0A90138
:100E6000082E02C0559547950A94E2F740FDCF5FE2
:100E700001968830910599F7C13061F0C23031F1A7
:100E8000EFEFEE1AFE0AF2E2EF16F0E0FF06F9F6D7
:100E9000C0E0BFCFDA11F4CFD12CC12C092110E072
:100EA000C8010C2C02C0959587950A94E2F780FF43
:100EB00014C08C2D31DFE82FF0E0EA58FF4F80811D
:100EC000823059F4809169008083A3CFD230C1F67B
:100ED0008091690080937A009BCFFFEFCF1ADF0AE1
:100EE00088E0C816D104E1F6CBCFDF92EF92FF92F3
:100EF0000F931F93CF93DF9380916A0015DFD82E55
:100F0000D0E0C0E0FE01E354FE4FE4918D2D8E232E
:100F10008E132BC0FE01E254FE4FE49110E000E07E
:100F2000EE2EF12CC701002E02C0959587950A94EC
:100F3000E2F780FF15C0802FEFDEE82FF0E0EA58DF
:100F4000FF4F8081823061F480916900808381E06D
:100F5000DF91CF911F910F91FF90EF90DF90089557
:100F60000F5F1F4F08301105E9F62296C032D105F8
:100F700049F680E0EDCFCF92DF92EF92FF920F9390
:100F8000CF93DF93F701C4913196E491A42FB0E0A1
:100F9000C82E880FDD08D0E0AE01415051094C0D3C
:100FA0005D1D4A175B078CF1AC15BD0574F1822FEE
:100FB00090E0062E000C770B8617970734F1F0E0CF
:100FC0009F0121503109260F371F28173907ECF0F0
:100FD000861B970BBE010DD7AC19BD09A80FB91F11
:100FE000CE01BF0106D7602F70E003D7FD01E80FE7
:100FF000F91F3296EE0DFF1D8491DF91CF910F9175
:10100000FF90EF90DF90CF90089580E0F6CFEF92C1
:10101000FF920F931F93CF93DF93C82FD62F86E2B3
:10102000E82E80E0F82E00916700262F4C2F60E01C
:1010300089E1A1DF182F009166002D2F4C2F60E071
:101040008AE599DF812BDF91CF911F910F91FF905E
:10105000EF9008955F926F927F928F929F92AF92DE
:10106000BF92CF92DF92EF92FF920F931F93CF9395
:10107000DF93762E813009F043C01092800060909B
:101080007F0061106090800060928000072D10E06A
:10109000C80162E170E0ADD684976C01C80164E2DA
:1010A00070E0A7D6845B91097C011695102F00276C
:1010B0001795079580EB870DBCDD80E0BADD80E1F8
:1010C000B8DDC2DDD0E0C0E0C80181509F4F5C01B7
:1010D000C80181509B4F4C019C2FC038D10509F4A9
:1010E000E4C081E08715A0F0F401EC0FFD1F5490DF
:1010F000672D8C2F8CDF8095482F452180E060C0C4
:1011000081E090918000911180E080938000B7CFC2
:10111000F501EC0FFD1F449184E0781609F454C0EA
:10112000871560F082E0781648F3CA34A0F4C8331B
:1011300048F59452923110F790E011C086E087157F
:10114000E8F2C23508F07CC0CF3208F090C0CB3056
:10115000A8F290E079C09B54923180F692E0292F5A
:1011600030E0F901EA58FF4F808150917400591323
:101170000BC090917500911107C091E0691207C0F2
:1011800082E005C091E0EBCF823009F4B7CFF901DE
:10119000ED5BF84F549090E06CE670E02AD6FC01CD
:1011A000C90164E270E025D6E80FF91FCE01851968
:1011B0009109E80FF91FEC0DFD1DE150FA4F8491E4
:1011C000842B19DD219688CFCE3440F4C433E0F46B
:1011D00099519A3108F092CF90E004C0C83608F0D7
:1011E0008DCF92E0A92FB0E0FD01EA58FF4F838137
:1011F0002091740029130AC090917500913031F448
:10120000691207C082E005C091E0ECCF823009F49A
:1012100075CFFD01E05DF74F549090E06EE470E013
:10122000E8D5FC01CD016AE170E0E3D5E80FF91FD4
:10123000CE0185199109E80FF91FEA5BF84FBFCF7E
:10124000C63708F05BCF92E0A92FB0E0FD01EA5865
:10125000FF4F86812091740092130BC0909175000E
:10126000923039F491E0691207C082E005C091E044
:10127000EBCF823009F442CFFD01E554F54F549095
:1012800090E068ED70E0B5D5FC01CD0168E470E058
:10129000B0D5E80FF91FCE0185199109E80FF91FA4
:1012A000EE0DFF1DED5CF74F8ACFA0DC739482E159
:1012B000C80ED11C94E2E90EF11C00581F4F88E0C3
:1012C0007812F8CEDF91CF911F910F91FF90EF90A0
:1012D000DF90CF90BF90AF909F908F907F906F9056
:1012E0005F90089560E081E0B5CE6F927F928F921B
:1012F0009F92AF92BF92CF92DF92EF92FF920F93A5
:101300001F93CF93DF9300D01F92CDB7DEB7682E27
:10131000B12CA12CAB8280EB8A0D8BDC80E089DCC8
:1013200080E187DC91DCD12CC12CC5019695982FEA
:101330008827979587959C0121503B4F49013B8118
:10134000335039837C2C80E8C816D10409F440C09E
:101350009B81923078F029812330C0F580E5E82E1A
:1013600080E0F82E00E02B814C2D63E086E303DE65
:101370008A830CC0F401EC0DFD1D34913A836B811E
:101380008C2D45DE80959A8198239A830DE511E096
:101390002B81472D662D84E3AEDB2A81282B2A83FF
:1013A0000EE810E02B81472D63E188E0A4DB3A8151
:1013B000382B3A832B81472D63E180E59CDB9A81B2
:1013C000892B19DC2FEFC21AD20ABCCF1A82DECFCA
:1013D0000DDC3FEFA31AB30A88E0A816B10409F0A8
:1013E00099CF0F900F900F90DF91CF911F910F9198
:1013F000FF90EF90DF90CF90BF90AF909F908F9035
:101400007F906F90089590E02FEF30E0281B310916
:101410008111C49A40E04217130634F455E05A95FE
:10142000F1F700004F5FF7CFC49840E04217130672
:1014300034F455E05A95F1F700004F5FF7CF9F5F06
:101440006913E6CF0895CF93CEE164E08AE0DBDF55
:101450008FE79EE30197F1F700C0000064E084E6A7
:10146000D2DFC15091F782E08093760080937700BD
:10147000809378008093790080937A0080937B003A
:1014800080937C0080937D0080937E0010927F008B
:10149000CF9128CFCF93DF938730E0F4E82FF0E0AF
:1014A000ED5AF54F099419C005C01FC021C023C0D3
:1014B0002CC038C0C0E064E08C2FA5DFC65FC43606
:1014C000D1F72FEF80E792E0215080409040E1F784
:1014D00000C00000DF91CF910895C4E663E08C2F37
:1014E00092DFC65FC83CD1F7ECCFDF91CF9122C02D
:1014F000DF91CF91A8CFC3E160E584E084DF60E5B0
:1015000084E681DFC150C1F7E5CFC8ECD8EC63E0D9
:101510008D2F8C1B78DF6CE08C2F75DFC150CA30AB
:10152000B1F7D8CF6AEF84E66EDF6AEF84E1DF912E
:10153000CF9169CFCF92DF92EF92FF920F931F93DB
:10154000CF93DF93CDB7DEB729970FB6F894DEBF00
:101550000FBECDBFFE01319606E710E0D8018D9198
:101560008D018193B0E00F371B07C1F78AE0D82EB9
:1015700092E0C92EEE24E394F12CEC0EFD1E89E0DE
:10158000E80EF11C6AE08CE83EDF64E08CED3BDFA6
:10159000E0917F00F0E0E759FF4F8081E6E7F0E05F
:1015A0009191981303C0DF011197CC920E171F077A
:1015B000B9F798DEA6E7B0E0FE01319681918D93F0
:1015C000EE15FF05D9F764E08AE01DDF8BDEDA94C3
:1015D000D110D8CF12E010937600109377001093BB
:1015E00078001093790010937A0010937B00109389
:1015F0007C0010937D0010937E0080917F008823F3
:1016000021F0813019F110E00EC080916600893020
:1016100020F48F5F80936600F6CF85E03BDF81E0AA
:101620008093680011E010927F005CDE812F299684
:101630000FB6F894DEBF0FBECDBFDF91CF911F91E3
:101640000F91FF90EF90DF90CF9008958091670009
:10165000893020F48F5F80936700D5CF84E01ADF54
:1016600010936800DFCFFF920F931F93CF93DF9308
:10167000082F5ADBF82ECEE1D0E010E0FE01849175
:1016800094918F218917C1F01F5F21961830B1F70F
:10169000E6E7F0E02FE730E080E09191923009F446
:1016A00081E02E173F07C9F781110FC0DF91CF915D
:1016B0001F910F91FF90C7CE143020F480917A00D3
:1016C0008013E2CF37DF8823F9F2DF91CF911F91AA
:1016D0000F91FF9008951F920F920FB60F92112451
:1016E0002F933F938F939F93AF93BF9380917000FD
:1016F00090917100A0917200B091730030916F00D1
:1017000023E0230F2D3768F126E8230F0296A11D51
:10171000B11D20936F008093700090937100A0938F
:101720007200B093730080916B0090916C00A09157
:101730006D00B0916E000196A11DB11D80936B00EC
:1017400090936C00A0936D00B0936E00BF91AF9129
:101750009F918F913F912F910F900FBE0F901F90EF
:1017600018950196A11DB11DD4CF83E08ABD83BF1A
:10177000789489B7826089BF80E48CBD8FEF8DBD7E
:1017800087EC80BF86B1876886B9379AB89ABA9ACB
:10179000CDE9D1E009EB11E0FE0184914ADA21960E
:1017A0000C171D07C9F760E081E06CDA61E084E0A6
:1017B00069DA60E080E866DA60E083E863DAD1E065
:1017C00033E0E32EF12C44E0C42ED12C5CEB452E0B
:1017D00051E0552E6AEBA62E61E0B62E8091600096
:1017E00067E0FED28A5E81DD83E88CDA8E3E92402D
:1017F00084F183E887DA863B93405CF58FEF96E7C8
:10180000E1E081509040E040E1F700C0000083E853
:1018100079DA8E3E92409CF083E874DA863B9340FE
:1018200074F480916000823008F48F5F80936000D0
:1018300067E0D6D28A5E59DD63E088ECE4DD83E8B8
:1018400061DA8E3E92402CF083E85CDA863B93406E
:10185000B4F383E857DA853F91407CF183E852DAAC
:101860008E3E924054F5FFEF26E781E0F150204094
:101870008040E1F700C0000083E844DA853F9140F2
:1018800094F083E83FDA8E3E92406CF480916000E1
:10189000811181508093600067E0A2D28A5E25DDCD
:1018A00063E088ECB0DD83E82DDA853F91402CF0D1
:1018B00083E828DA8E3E9240B4F3CBD9892B09F025
:1018C00093CFC7D90197E9F7D0937F0010926800B2
:1018D0001092670010926600D0937400D093750048
:1018E00082E08093760080937700809378008093E5
:1018F000790080937A0080937B0080937C008093B2
:101900007D0080937E0010926900D0936A0060E0B1
:1019100080E0A0DB86E0BEDDFFEF29E688E1F15044
:1019200020408040E1F700C00000C0E080917F00CF
:10193000882309F4D1C080E8E5D9853F9140B4F50A
:1019400080E8E0D98E3E92400CF05CC083E8DAD9A2
:101950008E3E92400CF077C083E8D4D9853F914009
:101960000CF496C083E8CED98E3E92400CF090C025
:10197000FFEF26E781E0F15020408040E1F700C012
:10198000000083E8BFD9853F91400CF47FC083E815
:10199000B9D98E3E92400CF079C0C11123C080911C
:1019A0007500882309F46FC081506DC080E8AAD902
:1019B0008E3E92402CF6FFEF26E781E0F15020406A
:1019C0008040E1F700C0000080E89CD9853F91404D
:1019D0000CF45CC080E896D98E3E92400CF056C064
:1019E000CC2341F0C1E0809168008111F7CE62E024
:1019F00031DB9CCF80917400811181E08F5F8093F7
:101A00007400F0CF80E87ED9863B93400CF09ECFE7
:101A1000FFEF26E781E0F15020408040E1F700C071
:101A2000000080E86FD98E3E924084F180E86AD948
:101A3000863B93405CF5C111D5CF8091740088231B
:101A4000F1F28150DCCF83E85DD9863B93400CF006
:101A500083CF8FEF96E7E1E081509040E040E1F7DF
:101A600000C0000083E84ED98E3E92407CF083E8AF
:101A700049D9863B934054F4C111B4CF809175008D
:101A8000811181E08F5F80937500ACCFC111AACF27
:101A9000E0D8892B11F0C0E0A6CFE0917500F0E00E
:101AA0002091740030E0CF0163E070E0A2D18A5849
:101AB0009F4FDC01A20FB31F8C91823061F7C09160
:101AC0006A00FD01C0830EDC8C2FE4DC80916A008B
:101AD000CADD10927F0086CF70906900872D4ED9A5
:101AE00081110CC060906000662009F4A5C01091BF
:101AF0006A00812F43D9882309F4BAC0F3DB8091AF
:101B00006900C8DC80916900AEDDD0937F006BCFA7
:101B1000781244C0812F08D9382EE9EBF1E0849186
:101B2000932D9823981315C0F5010491912C812CC5
:101B300010E0C801082C02C0959587950A94E2F739
:101B400080FD5AC0FFEF8F1A9F0A28E08216910489
:101B500081F7EBEBF1E08491382283111FC0F20191
:101B60000491912C812C10E0C801082C02C095959D
:101B700087950A94E2F780FF0AC0882DCDD8E82F18
:101B8000F0E0EA58FF4F8081823009F43FC0FFEF58
:101B90008F1A9F0A28E08216910431F781E086159A
:101BA00008F04AC0A2D98111A9CF9FD98111A6CF2F
:101BB000B1D0B6012FD19927880F991F880F991F8F
:101BC000FC01E352FE4FA491B0E0AA58BF4F2C9104
:101BD000223051F0FC01E252FE4FA491B0E0AA582D
:101BE000BF4F2C912230A1F4E491F0E0EA58FF4F6E
:101BF00080916900808382CF882D8ED8E82FF0E015
:101C0000EA58FF4F8081823009F09CCF708276CFF6
:101C1000FC01E152FE4FA491B0E0AA58BF4F2C91B5
:101C2000223011F3FC01E052FE4FA491B0E0AA581B
:101C3000BF4F8C918230C1F26DD08C016BD0B70157
:101C4000E9D0FC01FF27C801B701E4D09C0133278C
:101C5000CF0163E070E0CDD08A589F4FDC01A20F26
:101C6000B31F8C91823041F780916900FD01C2CF92
:101C700080917A00823009F04BCF70927A003ECF8B
:101C80008F929F92AF92BF92CF92DF92EF92FF928C
:101C9000CF93DF93EC01688179818A819B81611503
:101CA00071058105910521F464E279ED8BE597E0FA
:101CB0002DE133EF41E050E055D049015A0127EAC8
:101CC00031E440E050E035D06B017C012CEE34EF84
:101CD0004FEF5FEFC501B4012CD0DC01CB018C0DBF
:101CE0009D1DAE1DBF1DB7FF03C00197A109B048E0
:101CF00088839983AA83BB839F77DF91CF91FF90DD
:101D0000EF90DF90CF90BF90AF909F908F9008950D
:101D1000B7DF089581E690E0B3DF0895B0E0A0E07A
:101D20008093610090936200A0936300B09364007D
:101D30000895EE27FF27AA27BB2708C0A20FB31FCD
:101D4000E41FF51F220F331F441F551F96958795DB
:101D50007795679598F37040A9F7009799F7BD01BB
:101D6000CF010895052E97FB16F400940FD057FD70
:101D700005D014D007FC02D046F408C05095409519
:101D8000309521953F4F4F4F5F4F08959095809527
:101D9000709561957F4F8F4F9F4F0895A1E21A2E46
:101DA000AA1BBB1BFD010DC0AA1FBB1FEE1FFF1FFF
:101DB000A217B307E407F50720F0A21BB30BE40B4F
:101DC000F50B661F771F881F991F1A9469F7609596
:101DD0007095809590959B01AC01BD01CF01089550
:101DE000002480FD060E660F11F08695D1F7802D38
:101DF00008950024552704C0080E591F880F991F05
:101E0000009729F076956795B8F37105B9F7802D9D
:101E1000952F089597FB072E16F4009406D077FDB2
:101E200008D00BD007FC05D03EF4909581959F4FCC
:101E30000895709561957F4F0895AA1BBB1B51E1D2
:101E400007C0AA1FBB1FA617B70710F0A61BB70B2A
:101E5000881F991F5A95A9F780959095BC01CD01CF
:061E60000895F894FFCF85
:061E660001010000000074
:00000001FF
